 w2k_lsa_auth

 Timestamp is 31dc0ebc (reproducible build file hash)

 Preferred load address is 0000000180000000

 Start         Length     Name                   Class
 0001:00000000 00002310H .text$mn                CODE
 0001:00002310 00000036H .text$mn$00             CODE
 0001:00002346 00000092H .text$x                 CODE
 0002:00000000 000001b8H .idata$5                DATA
 0002:000001b8 00000038H .00cfg                  DATA
 0002:000001f0 00000008H .CRT$XCA                DATA
 0002:000001f8 00000008H .CRT$XCZ                DATA
 0002:00000200 00000008H .CRT$XIA                DATA
 0002:00000208 00000008H .CRT$XIZ                DATA
 0002:00000210 00000008H .CRT$XPA                DATA
 0002:00000218 00000008H .CRT$XPZ                DATA
 0002:00000220 00000008H .CRT$XTA                DATA
 0002:00000228 00000008H .CRT$XTZ                DATA
 0002:00000230 00000000H .gehcont$y              DATA
 0002:00000230 00000000H .gfids$y                DATA
 0002:00000230 00000dd0H .rdata                  DATA
 0002:00001000 00000000H .rdata$CastGuardVftablesA DATA
 0002:00001000 00000000H .rdata$CastGuardVftablesC DATA
 0002:00001000 0000006cH .rdata$voltmd           DATA
 0002:0000106c 000002bcH .rdata$zzzdbg           DATA
 0002:00001328 00000008H .rtc$IAA                DATA
 0002:00001330 00000008H .rtc$IZZ                DATA
 0002:00001338 00000008H .rtc$TAA                DATA
 0002:00001340 00000008H .rtc$TZZ                DATA
 0002:00001348 000002a8H .xdata                  DATA
 0002:000015f0 000000e8H .edata                  DATA
 0002:000016d8 000000a0H .idata$2                DATA
 0002:00001778 00000018H .idata$3                DATA
 0002:00001790 000001b8H .idata$4                DATA
 0002:00001948 0000048aH .idata$6                DATA
 0003:00000000 00000040H .data                   DATA
 0003:00000040 00000878H .bss                    DATA
 0004:00000000 00000288H .pdata                  DATA
 0005:00000000 00000060H .rsrc$01                DATA
 0005:00000060 00000328H .rsrc$02                DATA

  Address         Publics by Value              Rva+Base               Lib:Object

 0000:00000000       __AbsoluteZero             0000000000000000     <absolute>
 0000:00000000       ___safe_se_handler_count   0000000000000000     <absolute>
 0000:00000000       ___safe_se_handler_table   0000000000000000     <absolute>
 0000:00000000       __arm64x_extra_rfe_table   0000000000000000     <absolute>
 0000:00000000       __arm64x_extra_rfe_table_size 0000000000000000     <absolute>
 0000:00000000       __arm64x_native_entrypoint 0000000000000000     <absolute>
 0000:00000000       __arm64x_redirection_metadata 0000000000000000     <absolute>
 0000:00000000       __arm64x_redirection_metadata_count 0000000000000000     <absolute>
 0000:00000000       __dynamic_value_reloc_table 0000000000000000     <absolute>
 0000:00000000       __enclave_config           0000000000000000     <absolute>
 0000:00000000       __guard_check_icall_a64n_fptr 0000000000000000     <absolute>
 0000:00000000       __guard_eh_cont_count      0000000000000000     <absolute>
 0000:00000000       __guard_eh_cont_table      0000000000000000     <absolute>
 0000:00000000       __guard_fids_count         0000000000000000     <absolute>
 0000:00000000       __guard_fids_table         0000000000000000     <absolute>
 0000:00000000       __guard_iat_count          0000000000000000     <absolute>
 0000:00000000       __guard_iat_table          0000000000000000     <absolute>
 0000:00000000       __guard_longjmp_count      0000000000000000     <absolute>
 0000:00000000       __guard_longjmp_table      0000000000000000     <absolute>
 0000:00000000       __hybrid_auxiliary_delayload_iat 0000000000000000     <absolute>
 0000:00000000       __hybrid_auxiliary_delayload_iat_copy 0000000000000000     <absolute>
 0000:00000000       __hybrid_auxiliary_iat     0000000000000000     <absolute>
 0000:00000000       __hybrid_auxiliary_iat_copy 0000000000000000     <absolute>
 0000:00000000       __hybrid_code_map          0000000000000000     <absolute>
 0000:00000000       __hybrid_code_map_count    0000000000000000     <absolute>
 0000:00000000       __hybrid_image_info_bitfield 0000000000000000     <absolute>
 0000:00000000       __x64_code_ranges_to_entry_points 0000000000000000     <absolute>
 0000:00000000       __x64_code_ranges_to_entry_points_count 0000000000000000     <absolute>
 0000:00000100       __guard_flags              0000000000000100     <absolute>
 0000:00000000       __ImageBase                0000000180000000     <linker-defined>
 0001:00000000       BuildEncryptionKey         0000000180001000 f   NativeCreds.obj
 0001:000000e4       BuildKerberosTime          00000001800010e4 f   NativeCreds.obj
 0001:00000254       BuildPrincipal             0000000180001254 f   NativeCreds.obj
 0001:00000418       BuildTicket                0000000180001418 f   NativeCreds.obj
 0001:00000530       BuildTicketFlags           0000000180001530 f   NativeCreds.obj
 0001:000005e0       ConcatenateUnicodeStrings  00000001800015e0 f   NativeCreds.obj
 0001:0000072c       JNI_OnLoad                 000000018000172c f   NativeCreds.obj
 0001:00000cac       JNI_OnUnload               0000000180001cac f   NativeCreds.obj
 0001:00000d84       Java_sun_security_krb5_Credentials_acquireDefaultNativeCreds 0000000180001d84 f   NativeCreds.obj
 0001:000012a4       PackageConnectLookup       00000001800022a4 f   NativeCreds.obj
 0001:00001334       ShowLastError              0000000180002334 f   NativeCreds.obj
 0001:000013c8       ThrowOOME                  00000001800023c8 f   NativeCreds.obj
 0001:00001408       __local_stdio_printf_options 0000000180002408 f i NativeCreds.obj
 0001:00001410       printf                     0000000180002410 f i NativeCreds.obj
 0001:00001464       swprintf                   0000000180002464 f i NativeCreds.obj
 0001:000014b8       Java_sun_security_krb5_Config_getWindowsDirectory 00000001800024b8 f   WindowsDirectory.obj
 0001:00001528       LsaNtStatusToWinError      0000000180002528 f   advapi32:ADVAPI32.dll
 0001:0000152e       LsaLookupAuthenticationPackage 000000018000252e f   Secur32:Secur32.dll
 0001:00001534       LsaFreeReturnBuffer        0000000180002534 f   Secur32:Secur32.dll
 0001:0000153a       LsaCallAuthenticationPackage 000000018000253a f   Secur32:Secur32.dll
 0001:00001540       LsaConnectUntrusted        0000000180002540 f   Secur32:Secur32.dll
 0001:00001546       htonl                      0000000180002546 f   wsock32:WSOCK32.dll
 0001:0000154c       __GSHandlerCheck           000000018000254c f   MSVCRT:gshandler.obj
 0001:0000156c       __GSHandlerCheckCommon     000000018000256c f   MSVCRT:gshandler.obj
 0001:000015e0       __security_check_cookie    00000001800025e0 f   MSVCRT:amdsecgs.obj
 0001:00001920       _DllMainCRTStartup         0000000180002920 f   MSVCRT:dll_dllmain.obj
 0001:00001960       __raise_securityfailure    0000000180002960 f   MSVCRT:gs_report.obj
 0001:00001994       __report_gsfailure         0000000180002994 f   MSVCRT:gs_report.obj
 0001:00001adc       __security_init_cookie     0000000180002adc f   MSVCRT:gs_support.obj
 0001:00001b88       DllMain                    0000000180002b88 f   MSVCRT:dll_dllmain_stub.obj
 0001:00001bac       ?__scrt_initialize_type_info@@YAXXZ 0000000180002bac f   MSVCRT:tncleanup.obj
 0001:00001bbc       ?__scrt_uninitialize_type_info@@YAXXZ 0000000180002bbc f   MSVCRT:tncleanup.obj
 0001:00001bc8       __local_stdio_scanf_options 0000000180002bc8 f i MSVCRT:default_local_stdio_options.obj
 0001:00001bd0       __scrt_initialize_default_local_stdio_options 0000000180002bd0 f   MSVCRT:default_local_stdio_options.obj
 0001:00001bec       __scrt_acquire_startup_lock 0000000180002bec f   MSVCRT:utility.obj
 0001:00001c28       __scrt_dllmain_after_initialize_c 0000000180002c28 f   MSVCRT:utility.obj
 0001:00001c5c       __scrt_dllmain_before_initialize_c 0000000180002c5c f   MSVCRT:utility.obj
 0001:00001c74       __scrt_dllmain_crt_thread_attach 0000000180002c74 f   MSVCRT:utility.obj
 0001:00001c9c       __scrt_dllmain_crt_thread_detach 0000000180002c9c f   MSVCRT:utility.obj
 0001:00001cb4       __scrt_dllmain_exception_filter 0000000180002cb4 f   MSVCRT:utility.obj
 0001:00001d14       __scrt_dllmain_uninitialize_c 0000000180002d14 f   MSVCRT:utility.obj
 0001:00001d44       __scrt_dllmain_uninitialize_critical 0000000180002d44 f   MSVCRT:utility.obj
 0001:00001d58       __scrt_initialize_crt      0000000180002d58 f   MSVCRT:utility.obj
 0001:00001da4       __scrt_initialize_onexit_tables 0000000180002da4 f   MSVCRT:utility.obj
 0001:00001e30       __scrt_is_nonwritable_in_current_image 0000000180002e30 f   MSVCRT:utility.obj
 0001:00001ec8       __scrt_release_startup_lock 0000000180002ec8 f   MSVCRT:utility.obj
 0001:00001eec       __scrt_uninitialize_crt    0000000180002eec f   MSVCRT:utility.obj
 0001:00001f18       __scrt_get_dyn_tls_init_callback 0000000180002f18 f   MSVCRT:dyn_tls_init.obj
 0001:00001f20       __crt_debugger_hook        0000000180002f20 f   MSVCRT:utility_desktop.obj
 0001:00001f28       __scrt_fastfail            0000000180002f28 f   MSVCRT:utility_desktop.obj
 0001:00002074       _RTC_Initialize            0000000180003074 f   MSVCRT:initsect.obj
 0001:000020b0       _RTC_Terminate             00000001800030b0 f   MSVCRT:initsect.obj
 0001:000020ec       _guard_check_icall_nop     00000001800030ec f i MSVCRT:guard_support.obj
 0001:000020f0       __isa_available_init       00000001800030f0 f   MSVCRT:cpu_disp.obj
 0001:0000229c       _get_startup_argv_mode     000000018000329c f   MSVCRT:argv_mode.obj
 0001:000022a4       __scrt_is_ucrt_dll_in_use  00000001800032a4 f   MSVCRT:ucrt_detection.obj
 0001:000022b0       memcpy                     00000001800032b0 f   vcruntime:VCRUNTIME140.dll
 0001:000022b6       __C_specific_handler       00000001800032b6 f   vcruntime:VCRUNTIME140.dll
 0001:000022bc       __std_type_info_destroy_list 00000001800032bc f   vcruntime:VCRUNTIME140.dll
 0001:000022c2       memset                     00000001800032c2 f   vcruntime:VCRUNTIME140.dll
 0001:000022c8       strlen                     00000001800032c8 f   ucrt:api-ms-win-crt-string-l1-1-0.dll
 0001:000022ce       _initterm                  00000001800032ce f   ucrt:api-ms-win-crt-runtime-l1-1-0.dll
 0001:000022d4       _initterm_e                00000001800032d4 f   ucrt:api-ms-win-crt-runtime-l1-1-0.dll
 0001:000022da       _seh_filter_dll            00000001800032da f   ucrt:api-ms-win-crt-runtime-l1-1-0.dll
 0001:000022e0       _configure_narrow_argv     00000001800032e0 f   ucrt:api-ms-win-crt-runtime-l1-1-0.dll
 0001:000022e6       _initialize_narrow_environment 00000001800032e6 f   ucrt:api-ms-win-crt-runtime-l1-1-0.dll
 0001:000022ec       _initialize_onexit_table   00000001800032ec f   ucrt:api-ms-win-crt-runtime-l1-1-0.dll
 0001:000022f2       _execute_onexit_table      00000001800032f2 f   ucrt:api-ms-win-crt-runtime-l1-1-0.dll
 0001:000022f8       _cexit                     00000001800032f8 f   ucrt:api-ms-win-crt-runtime-l1-1-0.dll
 0001:00002300       __acrt_initialize          0000000180003300 f   MSVCRT:ucrt_stubs.obj
 0001:00002300       __acrt_thread_attach       0000000180003300 f   MSVCRT:ucrt_stubs.obj
 0001:00002300       __acrt_thread_detach       0000000180003300 f   MSVCRT:ucrt_stubs.obj
 0001:00002300       __acrt_uninitialize        0000000180003300 f   MSVCRT:ucrt_stubs.obj
 0001:00002300       __acrt_uninitialize_critical 0000000180003300 f   MSVCRT:ucrt_stubs.obj
 0001:00002300       __scrt_stub_for_acrt_initialize 0000000180003300 f   MSVCRT:ucrt_stubs.obj
 0001:00002300       __scrt_stub_for_acrt_thread_attach 0000000180003300 f   MSVCRT:ucrt_stubs.obj
 0001:00002300       __scrt_stub_for_acrt_thread_detach 0000000180003300 f   MSVCRT:ucrt_stubs.obj
 0001:00002300       __scrt_stub_for_acrt_uninitialize 0000000180003300 f   MSVCRT:ucrt_stubs.obj
 0001:00002300       __scrt_stub_for_acrt_uninitialize_critical 0000000180003300 f   MSVCRT:ucrt_stubs.obj
 0001:00002300       __vcrt_initialize          0000000180003300 f   MSVCRT:ucrt_stubs.obj
 0001:00002300       __vcrt_thread_attach       0000000180003300 f   MSVCRT:ucrt_stubs.obj
 0001:00002300       __vcrt_thread_detach       0000000180003300 f   MSVCRT:ucrt_stubs.obj
 0001:00002300       __vcrt_uninitialize        0000000180003300 f   MSVCRT:ucrt_stubs.obj
 0001:00002300       __vcrt_uninitialize_critical 0000000180003300 f   MSVCRT:ucrt_stubs.obj
 0001:00002304       __scrt_stub_for_is_c_termination_complete 0000000180003304 f   MSVCRT:ucrt_stubs.obj
 0001:00002304       _is_c_termination_complete 0000000180003304 f   MSVCRT:ucrt_stubs.obj
 0001:00002320       _guard_dispatch_icall_nop  0000000180003320 f   MSVCRT:guard_dispatch.obj
 0001:00002340       _guard_xfg_dispatch_icall_nop 0000000180003340 f   MSVCRT:guard_xfg_dispatch.obj
 0002:00000000       __imp_LsaNtStatusToWinError 0000000180004000     advapi32:ADVAPI32.dll
 0002:00000008       \177ADVAPI32_NULL_THUNK_DATA 0000000180004008     advapi32:ADVAPI32.dll
 0002:00000010       __imp_IsDebuggerPresent    0000000180004010     kernel32:KERNEL32.dll
 0002:00000018       __imp_InitializeSListHead  0000000180004018     kernel32:KERNEL32.dll
 0002:00000020       __imp_DisableThreadLibraryCalls 0000000180004020     kernel32:KERNEL32.dll
 0002:00000028       __imp_GetCurrentThreadId   0000000180004028     kernel32:KERNEL32.dll
 0002:00000030       __imp_CompareFileTime      0000000180004030     kernel32:KERNEL32.dll
 0002:00000038       __imp_GetLastError         0000000180004038     kernel32:KERNEL32.dll
 0002:00000040       __imp_GetSystemTimeAsFileTime 0000000180004040     kernel32:KERNEL32.dll
 0002:00000048       __imp_LocalAlloc           0000000180004048     kernel32:KERNEL32.dll
 0002:00000050       __imp_LocalFree            0000000180004050     kernel32:KERNEL32.dll
 0002:00000058       __imp_FormatMessageW       0000000180004058     kernel32:KERNEL32.dll
 0002:00000060       __imp_FileTimeToSystemTime 0000000180004060     kernel32:KERNEL32.dll
 0002:00000068       __imp_GetWindowsDirectoryW 0000000180004068     kernel32:KERNEL32.dll
 0002:00000070       __imp_GetSystemWindowsDirectoryW 0000000180004070     kernel32:KERNEL32.dll
 0002:00000078       __imp_GetCurrentProcessId  0000000180004078     kernel32:KERNEL32.dll
 0002:00000080       __imp_QueryPerformanceCounter 0000000180004080     kernel32:KERNEL32.dll
 0002:00000088       __imp_IsProcessorFeaturePresent 0000000180004088     kernel32:KERNEL32.dll
 0002:00000090       __imp_TerminateProcess     0000000180004090     kernel32:KERNEL32.dll
 0002:00000098       __imp_GetCurrentProcess    0000000180004098     kernel32:KERNEL32.dll
 0002:000000a0       __imp_SetUnhandledExceptionFilter 00000001800040a0     kernel32:KERNEL32.dll
 0002:000000a8       __imp_UnhandledExceptionFilter 00000001800040a8     kernel32:KERNEL32.dll
 0002:000000b0       __imp_RtlVirtualUnwind     00000001800040b0     kernel32:KERNEL32.dll
 0002:000000b8       __imp_RtlLookupFunctionEntry 00000001800040b8     kernel32:KERNEL32.dll
 0002:000000c0       __imp_RtlCaptureContext    00000001800040c0     kernel32:KERNEL32.dll
 0002:000000c8       \177KERNEL32_NULL_THUNK_DATA 00000001800040c8     kernel32:KERNEL32.dll
 0002:000000d0       __imp_LsaCallAuthenticationPackage 00000001800040d0     Secur32:Secur32.dll
 0002:000000d8       __imp_LsaLookupAuthenticationPackage 00000001800040d8     Secur32:Secur32.dll
 0002:000000e0       __imp_LsaConnectUntrusted  00000001800040e0     Secur32:Secur32.dll
 0002:000000e8       __imp_LsaFreeReturnBuffer  00000001800040e8     Secur32:Secur32.dll
 0002:000000f0       \177Secur32_NULL_THUNK_DATA 00000001800040f0     Secur32:Secur32.dll
 0002:000000f8       __imp_memset               00000001800040f8     vcruntime:VCRUNTIME140.dll
 0002:00000100       __imp___C_specific_handler 0000000180004100     vcruntime:VCRUNTIME140.dll
 0002:00000108       __imp___std_type_info_destroy_list 0000000180004108     vcruntime:VCRUNTIME140.dll
 0002:00000110       __imp_memcpy               0000000180004110     vcruntime:VCRUNTIME140.dll
 0002:00000118       \177VCRUNTIME140_NULL_THUNK_DATA 0000000180004118     vcruntime:VCRUNTIME140.dll
 0002:00000120       __imp_htonl                0000000180004120     wsock32:WSOCK32.dll
 0002:00000128       \177WSOCK32_NULL_THUNK_DATA 0000000180004128     wsock32:WSOCK32.dll
 0002:00000130       __imp__initialize_onexit_table 0000000180004130     ucrt:api-ms-win-crt-runtime-l1-1-0.dll
 0002:00000138       __imp__execute_onexit_table 0000000180004138     ucrt:api-ms-win-crt-runtime-l1-1-0.dll
 0002:00000140       __imp__cexit               0000000180004140     ucrt:api-ms-win-crt-runtime-l1-1-0.dll
 0002:00000148       __imp__initialize_narrow_environment 0000000180004148     ucrt:api-ms-win-crt-runtime-l1-1-0.dll
 0002:00000150       __imp__configure_narrow_argv 0000000180004150     ucrt:api-ms-win-crt-runtime-l1-1-0.dll
 0002:00000158       __imp__seh_filter_dll      0000000180004158     ucrt:api-ms-win-crt-runtime-l1-1-0.dll
 0002:00000160       __imp__initterm_e          0000000180004160     ucrt:api-ms-win-crt-runtime-l1-1-0.dll
 0002:00000168       __imp__initterm            0000000180004168     ucrt:api-ms-win-crt-runtime-l1-1-0.dll
 0002:00000170       \177api-ms-win-crt-runtime-l1-1-0_NULL_THUNK_DATA 0000000180004170     ucrt:api-ms-win-crt-runtime-l1-1-0.dll
 0002:00000178       __imp___stdio_common_vswprintf 0000000180004178     ucrt:api-ms-win-crt-stdio-l1-1-0.dll
 0002:00000180       __imp___acrt_iob_func      0000000180004180     ucrt:api-ms-win-crt-stdio-l1-1-0.dll
 0002:00000188       __imp___stdio_common_vfprintf 0000000180004188     ucrt:api-ms-win-crt-stdio-l1-1-0.dll
 0002:00000190       \177api-ms-win-crt-stdio-l1-1-0_NULL_THUNK_DATA 0000000180004190     ucrt:api-ms-win-crt-stdio-l1-1-0.dll
 0002:00000198       __imp_wcslen               0000000180004198     ucrt:api-ms-win-crt-string-l1-1-0.dll
 0002:000001a0       __imp_strlen               00000001800041a0     ucrt:api-ms-win-crt-string-l1-1-0.dll
 0002:000001a8       __imp_wcsncpy              00000001800041a8     ucrt:api-ms-win-crt-string-l1-1-0.dll
 0002:000001b0       \177api-ms-win-crt-string-l1-1-0_NULL_THUNK_DATA 00000001800041b0     ucrt:api-ms-win-crt-string-l1-1-0.dll
 0002:000001b8       __guard_check_icall_fptr   00000001800041b8     MSVCRT:guard_support.obj
 0002:000001c0       __guard_xfg_check_icall_fptr 00000001800041c0     MSVCRT:guard_support.obj
 0002:000001c8       __guard_dispatch_icall_fptr 00000001800041c8     MSVCRT:guard_support.obj
 0002:000001d0       __guard_xfg_dispatch_icall_fptr 00000001800041d0     MSVCRT:guard_support.obj
 0002:000001d8       __guard_xfg_table_dispatch_icall_fptr 00000001800041d8     MSVCRT:guard_support.obj
 0002:000001e0       __castguard_check_failure_os_handled_fptr 00000001800041e0     MSVCRT:guard_support.obj
 0002:000001e8       __guard_memcpy_fptr        00000001800041e8     vcruntime:softmemtag.obj
 0002:000001f0       __xc_a                     00000001800041f0     MSVCRT:initializers.obj
 0002:000001f8       __xc_z                     00000001800041f8     MSVCRT:initializers.obj
 0002:00000200       __xi_a                     0000000180004200     MSVCRT:initializers.obj
 0002:00000208       __xi_z                     0000000180004208     MSVCRT:initializers.obj
 0002:00000210       __xp_a                     0000000180004210     MSVCRT:initializers.obj
 0002:00000218       __xp_z                     0000000180004218     MSVCRT:initializers.obj
 0002:00000220       __xt_a                     0000000180004220     MSVCRT:initializers.obj
 0002:00000228       __xt_z                     0000000180004228     MSVCRT:initializers.obj
 0002:00000230       ??_C@_0CA@MAAHMEAA@sun?1security?1krb5?1internal?1Krb5@ 0000000180004230     NativeCreds.obj
 0002:00000250       ??_C@_0BJ@ONBLC@LSA?3?5Couldn?8t?5find?5Krb5?6@ 0000000180004250     NativeCreds.obj
 0002:0000026c       ??_C@_01POHCFINO@Z@        000000018000426c     NativeCreds.obj
 0002:00000270       ??_C@_05KOLFGEDA@DEBUG@    0000000180004270     NativeCreds.obj
 0002:00000278       ??_C@_0BO@HKKMKLPH@LSA?3?5Krb5?5has?5no?5DEBUG?5field?6@ 0000000180004278     NativeCreds.obj
 0002:00000298       ??_C@_0CC@HHHDDMMJ@sun?1security?1krb5?1internal?1Tick@ 0000000180004298     NativeCreds.obj
 0002:000002c0       ??_C@_0BL@GBEIKIJJ@LSA?3?5Couldn?8t?5find?5Ticket?6@ 00000001800042c0     NativeCreds.obj
 0002:000002e0       ??_C@_0BD@NPHBGKOJ@LSA?3?5Found?5Ticket?6@ 00000001800042e0     NativeCreds.obj
 0002:000002f8       ??_C@_0BM@FJBDPNKL@LSA?3?5Made?5NewWeakGlobalRef?6@ 00000001800042f8     NativeCreds.obj
 0002:00000318       ??_C@_0CA@JFAAMJED@sun?1security?1krb5?1PrincipalName@ 0000000180004318     NativeCreds.obj
 0002:00000338       ??_C@_0CC@IGIMKEMM@LSA?3?5Couldn?8t?5find?5PrincipalNam@ 0000000180004338     NativeCreds.obj
 0002:00000360       ??_C@_0BK@GHFICIAG@LSA?3?5Found?5PrincipalName?6@ 0000000180004360     NativeCreds.obj
 0002:00000380       ??_C@_0BL@FEIPNCJB@sun?1security?1util?1DerValue@ 0000000180004380     NativeCreds.obj
 0002:000003a0       ??_C@_0BN@IMBPDDME@LSA?3?5Couldn?8t?5find?5DerValue?6@ 00000001800043a0     NativeCreds.obj
 0002:000003c0       ??_C@_0BF@NGEKFHJH@LSA?3?5Found?5DerValue?6@ 00000001800043c0     NativeCreds.obj
 0002:000003d8       ??_C@_0CA@PAIDIBIN@sun?1security?1krb5?1EncryptionKey@ 00000001800043d8     NativeCreds.obj
 0002:000003f8       ??_C@_0CC@PKDFMIDD@LSA?3?5Couldn?8t?5find?5EncryptionKe@ 00000001800043f8     NativeCreds.obj
 0002:00000420       ??_C@_0BK@BLOBEEPJ@LSA?3?5Found?5EncryptionKey?6@ 0000000180004420     NativeCreds.obj
 0002:00000440       ??_C@_0CH@CHOCOAEA@sun?1security?1krb5?1internal?1Tick@ 0000000180004440     NativeCreds.obj
 0002:00000468       ??_C@_0CA@EMAINPN@LSA?3?5Couldn?8t?5find?5TicketFlags?6@ 0000000180004468     NativeCreds.obj
 0002:00000488       ??_C@_0BI@HAKKBGJG@LSA?3?5Found?5TicketFlags?6@ 0000000180004488     NativeCreds.obj
 0002:000004a0       ??_C@_0CI@JKANDJAE@sun?1security?1krb5?1internal?1Kerb@ 00000001800044a0     NativeCreds.obj
 0002:000004c8       ??_C@_0CB@GDPEGAMP@LSA?3?5Couldn?8t?5find?5KerberosTime@ 00000001800044c8     NativeCreds.obj
 0002:000004f0       ??_C@_0BJ@LJOALCIE@LSA?3?5Found?5KerberosTime?6@ 00000001800044f0     NativeCreds.obj
 0002:00000510       ??_C@_0BB@FLFAIHG@java?1lang?1String@ 0000000180004510     NativeCreds.obj
 0002:00000528       ??_C@_0BL@BGKPEEPI@LSA?3?5Couldn?8t?5find?5String?6@ 0000000180004528     NativeCreds.obj
 0002:00000548       ??_C@_0BD@KIJGIGII@LSA?3?5Found?5String?6@ 0000000180004548     NativeCreds.obj
 0002:0000055c       ??_C@_05GBDANG@?$CI?$FLB?$CJV@ 000000018000455c     NativeCreds.obj
 0002:00000564       ??_C@_06FALKBLGB@?$DMinit?$DO@ 0000000180004564     NativeCreds.obj
 0002:00000570       ??_C@_0CJ@OMBJPAOB@LSA?3?5Couldn?8t?5find?5DerValue?5con@ 0000000180004570     NativeCreds.obj
 0002:000005a0       ??_C@_0CB@PPLABLED@LSA?3?5Found?5DerValue?5constructor@ 00000001800045a0     NativeCreds.obj
 0002:000005c8       ??_C@_0CA@ENJPEMDC@?$CILsun?1security?1util?1DerValue?$DL?$CJV@ 00000001800045c8     NativeCreds.obj
 0002:000005e8       ??_C@_0CH@CEEKCGJO@LSA?3?5Couldn?8t?5find?5Ticket?5const@ 00000001800045e8     NativeCreds.obj
 0002:00000610       ??_C@_0BP@ONIFIACG@LSA?3?5Found?5Ticket?5constructor?6@ 0000000180004610     NativeCreds.obj
 0002:00000630       ??_C@_0CJ@OCAKIDDP@?$CI?$FLLjava?1lang?1String?$DLLjava?1lang?1@ 0000000180004630     NativeCreds.obj
 0002:00000660       ??_C@_0CO@KFILNLLM@LSA?3?5Couldn?8t?5find?5PrincipalNam@ 0000000180004660     NativeCreds.obj
 0002:00000690       ??_C@_0CG@BJFEPGAO@LSA?3?5Found?5PrincipalName?5constr@ 0000000180004690     NativeCreds.obj
 0002:000006b8       ??_C@_06BDDFOFAP@?$CII?$FLB?$CJV@ 00000001800046b8     NativeCreds.obj
 0002:000006c0       ??_C@_0CO@KNCIDOBE@LSA?3?5Couldn?8t?5find?5EncryptionKe@ 00000001800046c0     NativeCreds.obj
 0002:000006f0       ??_C@_0CG@BBPHBDKG@LSA?3?5Found?5EncryptionKey?5constr@ 00000001800046f0     NativeCreds.obj
 0002:00000718       ??_C@_0CM@BLPDNPGC@LSA?3?5Couldn?8t?5find?5TicketFlags?5@ 0000000180004718     NativeCreds.obj
 0002:00000748       ??_C@_0CE@NDIPGHBE@LSA?3?5Found?5TicketFlags?5construc@ 0000000180004748     NativeCreds.obj
 0002:00000770       ??_C@_0BG@IKDDPPGD@?$CILjava?1lang?1String?$DL?$CJV@ 0000000180004770     NativeCreds.obj
 0002:00000788       ??_C@_0CN@FGFKFHHG@LSA?3?5Couldn?8t?5find?5KerberosTime@ 0000000180004788     NativeCreds.obj
 0002:000007b8       ??_C@_0CF@OPPEPPMH@LSA?3?5Found?5KerberosTime?5constru@ 00000001800047b8     NativeCreds.obj
 0002:000007e0       ??_C@_0CB@CGFFPHE@LSA?3?5Finished?5OnLoad?5processing@ 00000001800047e0     NativeCreds.obj
 0002:00000810       ??_C@_0BMC@HPGKICPC@?$CILsun?1security?1krb5?1internal?1Ti@ 0000000180004810     NativeCreds.obj
 0002:000009d8       ??_C@_0DO@EFFGMMEG@LSA?3?5Couldn?8t?5find?5sun?4security@ 00000001800049d8     NativeCreds.obj
 0002:00000a18       ??_C@_0CB@EHGDGLDH@LSA?3?5Found?5KrbCreds?5constructor@ 0000000180004a18     NativeCreds.obj
 0002:00000a40       ??_C@_0CF@LMFMNKOO@LSA?3?5Got?5handle?5to?5Kerberos?5pac@ 0000000180004a40     NativeCreds.obj
 0002:00000a68       ??_C@_0BK@LHGHINFG@LSA?3?5Response?5size?5is?5?$CFd?6@ 0000000180004a68     NativeCreds.obj
 0002:00000a88       ??_C@_0BN@HFCMCMJP@LsaCallAuthenticationPackage@ 0000000180004a88     NativeCreds.obj
 0002:00000aa8       ??_C@_0BA@HOOKBKLM@Protocol?5status@ 0000000180004aa8     NativeCreds.obj
 0002:00000ab8       ??_C@_0CG@BNMCCPEA@LSA?3?5TICKET?5SessionKey?5KeyType?5@ 0000000180004ab8     NativeCreds.obj
 0002:00000ae0       ??_C@_0BM@PMFBHKAH@LSA?3?5Valid?5etype?5found?3?5?$CFd?6@ 0000000180004ae0     NativeCreds.obj
 0002:00000b00       ??_C@_0ED@ENPOMDNM@LSA?3?5MS?5TGT?5in?5cache?5is?5invalid@ 0000000180004b00     NativeCreds.obj
 0002:00000b48       ??_C@_0BO@JMBJFFMC@ConstructTicketRequest?5status@ 0000000180004b48     NativeCreds.obj
 0002:00000b68       ??_C@_0CB@JAMPMMEM@LSA?3?5Response?5size?5is?5?$CFd?5for?5?$CFd@ 0000000180004b68     NativeCreds.obj
 0002:00000b90       ??_C@_0CK@NMHODGIB@LSA?3?5Response?5etype?5is?5?$CFd?5for?5?$CF@ 0000000180004b90     NativeCreds.obj
 0002:00000bc0       ??_C@_1BA@PCNIOLBA@?$AAk?$AAr?$AAb?$AAt?$AAg?$AAt?$AA?1@ 0000000180004bc0     NativeCreds.obj
 0002:00000bd0       ??_C@_0CB@EAICCFNK@Can?8t?5allocate?5memory?5for?5ticke@ 0000000180004bd0     NativeCreds.obj
 0002:00000bf8       ??_C@_0BE@EAEONKAL@LsaConnectUntrusted@ 0000000180004bf8     NativeCreds.obj
 0002:00000c10       ??_C@_08DEIMIBAF@Kerberos@ 0000000180004c10     NativeCreds.obj
 0002:00000c20       ??_C@_0BP@OOIEHDKO@LsaLookupAuthenticationPackage@ 0000000180004c20     NativeCreds.obj
 0002:00000c40       ??_C@_0CF@EDKDHEBD@LSA?3?5Error?5calling?5function?5?$CFs?3@ 0000000180004c40     NativeCreds.obj
 0002:00000c68       ??_C@_0CD@FALAEFFE@LSA?3?5FormatMessage?5failed?5with?5@ 0000000180004c68     NativeCreds.obj
 0002:00000c90       ??_C@_07NGGFFIFC@LSA?3?5?$CFS@ 0000000180004c90     NativeCreds.obj
 0002:00000c98       ??_C@_0CA@HOHAFDNF@Can?8t?5allocate?5memory?5for?5realm@ 0000000180004c98     NativeCreds.obj
 0002:00000cb8       ??_C@_0BN@GMKMIDMN@LSA?3?5Principal?5domain?5is?5?$CFS?6@ 0000000180004cb8     NativeCreds.obj
 0002:00000cd8       ??_C@_0BG@KJEAEOON@LSA?3?5Name?5type?5is?5?$CFx?6@ 0000000180004cd8     NativeCreds.obj
 0002:00000cf0       ??_C@_0BH@HBDBBNHO@LSA?3?5Name?5count?5is?5?$CFx?6@ 0000000180004cf0     NativeCreds.obj
 0002:00000d08       ??_C@_0DA@HIADNNPN@LSA?3?5Can?8t?5allocate?5String?5arra@ 0000000180004d08     NativeCreds.obj
 0002:00000d38       ??_C@_0CC@JPDKOOFK@LSA?3?5Session?5key?5all?5zero?4?5Stop@ 0000000180004d38     NativeCreds.obj
 0002:00000d60       ??_C@_1M@HJLEHBOL@?$AA?$CF?$AA2?$AA?4?$AA2?$AAd@ 0000000180004d60     NativeCreds.obj
 0002:00000d70       ??_C@_1EG@KKOCIAIL@?$AA?$CF?$AAl?$AAd?$AA?$CF?$AA0?$AA2?$AA?4?$AA2?$AAs?$AA?$CF?$AA0?$AA2?$AA?4?$AA2?$AAs@ 0000000180004d70     NativeCreds.obj
 0002:00000db8       ??_C@_08HPFMLNAK@LSA?3?5?$CFS?6@ 0000000180004db8     NativeCreds.obj
 0002:00000dc8       ??_C@_0BL@ENCPOIKC@java?1lang?1OutOfMemoryError@ 0000000180004dc8     NativeCreds.obj
 0002:00000de8       _pDefaultRawDllMain        0000000180004de8     MSVCRT:dll_dllmain.obj
 0002:00000de8       _pRawDllMain               0000000180004de8     MSVCRT:dll_dllmain.obj
 0002:00000e00       __xmm@ffffffffffffffffffffffffffffffff 0000000180004e00     MSVCRT:utility.obj
 0002:00000e10       _load_config_used          0000000180004e10     MSVCRT:loadcfg.obj
 0002:00001000       __volatile_metadata        0000000180005000     <linker-defined>
 0002:00001328       __rtc_iaa                  0000000180005328     MSVCRT:initsect.obj
 0002:00001330       __rtc_izz                  0000000180005330     MSVCRT:initsect.obj
 0002:00001338       __rtc_taa                  0000000180005338     MSVCRT:initsect.obj
 0002:00001340       __rtc_tzz                  0000000180005340     MSVCRT:initsect.obj
 0002:000016d8       __IMPORT_DESCRIPTOR_ADVAPI32 00000001800056d8     advapi32:ADVAPI32.dll
 0002:000016ec       __IMPORT_DESCRIPTOR_Secur32 00000001800056ec     Secur32:Secur32.dll
 0002:00001700       __IMPORT_DESCRIPTOR_KERNEL32 0000000180005700     kernel32:KERNEL32.dll
 0002:00001714       __IMPORT_DESCRIPTOR_WSOCK32 0000000180005714     wsock32:WSOCK32.dll
 0002:00001728       __IMPORT_DESCRIPTOR_VCRUNTIME140 0000000180005728     vcruntime:VCRUNTIME140.dll
 0002:0000173c       __IMPORT_DESCRIPTOR_api-ms-win-crt-string-l1-1-0 000000018000573c     ucrt:api-ms-win-crt-string-l1-1-0.dll
 0002:00001750       __IMPORT_DESCRIPTOR_api-ms-win-crt-stdio-l1-1-0 0000000180005750     ucrt:api-ms-win-crt-stdio-l1-1-0.dll
 0002:00001764       __IMPORT_DESCRIPTOR_api-ms-win-crt-runtime-l1-1-0 0000000180005764     ucrt:api-ms-win-crt-runtime-l1-1-0.dll
 0002:00001778       __NULL_IMPORT_DESCRIPTOR   0000000180005778     advapi32:ADVAPI32.dll
 0003:00000000       __security_cookie_complement 0000000180006000     MSVCRT:gs_cookie.obj
 0003:00000008       __security_cookie          0000000180006008     MSVCRT:gs_cookie.obj
 0003:00000010       __scrt_native_dllmain_reason 0000000180006010     MSVCRT:utility.obj
 0003:00000018       __isa_available            0000000180006018     MSVCRT:cpu_disp.obj
 0003:0000001c       __isa_enabled              000000018000601c     MSVCRT:cpu_disp.obj
 0003:00000020       __memset_fast_string_threshold 0000000180006020     MSVCRT:cpu_disp.obj
 0003:00000028       __memset_nt_threshold      0000000180006028     MSVCRT:cpu_disp.obj
 0003:00000030       __scrt_ucrt_dll_is_in_use  0000000180006030     MSVCRT:ucrt_stubs.obj
 0003:00000040       derValueClass              0000000180006040     NativeCreds.obj
 0003:00000048       ticketClass                0000000180006048     NativeCreds.obj
 0003:00000050       principalNameClass         0000000180006050     NativeCreds.obj
 0003:00000058       encryptionKeyClass         0000000180006058     NativeCreds.obj
 0003:00000060       ticketFlagsClass           0000000180006060     NativeCreds.obj
 0003:00000068       kerberosTimeClass          0000000180006068     NativeCreds.obj
 0003:00000070       javaLangStringClass        0000000180006070     NativeCreds.obj
 0003:00000078       derValueConstructor        0000000180006078     NativeCreds.obj
 0003:00000080       ticketConstructor          0000000180006080     NativeCreds.obj
 0003:00000088       principalNameConstructor   0000000180006088     NativeCreds.obj
 0003:00000090       encryptionKeyConstructor   0000000180006090     NativeCreds.obj
 0003:00000098       ticketFlagsConstructor     0000000180006098     NativeCreds.obj
 0003:000000a0       kerberosTimeConstructor    00000001800060a0     NativeCreds.obj
 0003:000000a8       krbcredsConstructor        00000001800060a8     NativeCreds.obj
 0003:000000b0       native_debug               00000001800060b0     NativeCreds.obj
 0003:00000840       ?__type_info_root_node@@3U__type_info_node@@A 0000000180006840     MSVCRT:tncleanup.obj
 0003:00000850       ?_OptionsStorage@?1??__local_stdio_scanf_options@@9@4_KA 0000000180006850     MSVCRT:default_local_stdio_options.obj
 0003:00000858       __scrt_current_native_startup_state 0000000180006858     MSVCRT:utility.obj
 0003:00000860       __scrt_native_startup_lock 0000000180006860     MSVCRT:utility.obj
 0003:000008a0       __scrt_debugger_hook_flag  00000001800068a0     MSVCRT:utility_desktop.obj
 0003:000008a4       __favor                    00000001800068a4     MSVCRT:cpu_disp.obj
 0003:000008a8       ?_OptionsStorage@?1??__local_stdio_printf_options@@9@9 00000001800068a8     <common>
 0003:000008b0       __dyn_tls_init_callback    00000001800068b0     <common>

 entry point at        0001:00001920

 Static symbols

 0000:ffff6000       .debug$S                   0000000180000000     w2k_lsa_auth.exp
 0000:ffff6000       .debug$S                   0000000180000000     vcruntime:VCRUNTIME140.dll
 0000:ffff6000       .debug$S                   0000000180000000     vcruntime:VCRUNTIME140.dll
 0000:ffff6000       .debug$S                   0000000180000000     vcruntime:VCRUNTIME140.dll
 0000:ffff6000       .debug$S                   0000000180000000     vcruntime:VCRUNTIME140.dll
 0000:ffff6000       .debug$S                   0000000180000000     vcruntime:VCRUNTIME140.dll
 0000:ffff6000       .debug$S                   0000000180000000     vcruntime:VCRUNTIME140.dll
 0000:ffff6000       .debug$S                   0000000180000000     ucrt:api-ms-win-crt-runtime-l1-1-0.dll
 0000:ffff6000       .debug$S                   0000000180000000     ucrt:api-ms-win-crt-runtime-l1-1-0.dll
 0000:ffff6000       .debug$S                   0000000180000000     ucrt:api-ms-win-crt-runtime-l1-1-0.dll
 0000:ffff6000       .debug$S                   0000000180000000     ucrt:api-ms-win-crt-runtime-l1-1-0.dll
 0000:ffff6000       .debug$S                   0000000180000000     ucrt:api-ms-win-crt-runtime-l1-1-0.dll
 0000:ffff6000       .debug$S                   0000000180000000     ucrt:api-ms-win-crt-runtime-l1-1-0.dll
 0000:ffff6000       .debug$S                   0000000180000000     ucrt:api-ms-win-crt-runtime-l1-1-0.dll
 0000:ffff6000       .debug$S                   0000000180000000     ucrt:api-ms-win-crt-runtime-l1-1-0.dll
 0000:ffff6000       .debug$S                   0000000180000000     ucrt:api-ms-win-crt-runtime-l1-1-0.dll
 0000:ffff6000       .debug$S                   0000000180000000     ucrt:api-ms-win-crt-runtime-l1-1-0.dll
 0000:ffff6000       .debug$S                   0000000180000000     ucrt:api-ms-win-crt-runtime-l1-1-0.dll
 0000:ffff6000       .debug$S                   0000000180000000     ucrt:api-ms-win-crt-runtime-l1-1-0.dll
 0000:ffff6000       .debug$S                   0000000180000000     ucrt:api-ms-win-crt-stdio-l1-1-0.dll
 0000:ffff6000       .debug$S                   0000000180000000     ucrt:api-ms-win-crt-stdio-l1-1-0.dll
 0000:ffff6000       .debug$S                   0000000180000000     ucrt:api-ms-win-crt-stdio-l1-1-0.dll
 0000:ffff6000       .debug$S                   0000000180000000     ucrt:api-ms-win-crt-string-l1-1-0.dll
 0000:ffff6000       .debug$S                   0000000180000000     ucrt:api-ms-win-crt-string-l1-1-0.dll
 0000:ffff6000       .debug$S                   0000000180000000     ucrt:api-ms-win-crt-string-l1-1-0.dll
 0000:ffff6000       .debug$S                   0000000180000000     Secur32:Secur32.dll
 0000:ffff6000       .debug$S                   0000000180000000     Secur32:Secur32.dll
 0000:ffff6000       .debug$S                   0000000180000000     Secur32:Secur32.dll
 0000:ffff6000       .debug$S                   0000000180000000     Secur32:Secur32.dll
 0000:ffff6000       .debug$S                   0000000180000000     advapi32:ADVAPI32.dll
 0000:ffff6000       .debug$S                   0000000180000000     kernel32:KERNEL32.dll
 0000:ffff6000       .debug$S                   0000000180000000     kernel32:KERNEL32.dll
 0000:ffff6000       .debug$S                   0000000180000000     kernel32:KERNEL32.dll
 0000:ffff6000       .debug$S                   0000000180000000     kernel32:KERNEL32.dll
 0000:ffff6000       .debug$S                   0000000180000000     kernel32:KERNEL32.dll
 0000:ffff6000       .debug$S                   0000000180000000     kernel32:KERNEL32.dll
 0000:ffff6000       .debug$S                   0000000180000000     kernel32:KERNEL32.dll
 0000:ffff6000       .debug$S                   0000000180000000     kernel32:KERNEL32.dll
 0000:ffff6000       .debug$S                   0000000180000000     kernel32:KERNEL32.dll
 0000:ffff6000       .debug$S                   0000000180000000     kernel32:KERNEL32.dll
 0000:ffff6000       .debug$S                   0000000180000000     kernel32:KERNEL32.dll
 0000:ffff6000       .debug$S                   0000000180000000     kernel32:KERNEL32.dll
 0000:ffff6000       .debug$S                   0000000180000000     kernel32:KERNEL32.dll
 0000:ffff6000       .debug$S                   0000000180000000     kernel32:KERNEL32.dll
 0000:ffff6000       .debug$S                   0000000180000000     kernel32:KERNEL32.dll
 0000:ffff6000       .debug$S                   0000000180000000     kernel32:KERNEL32.dll
 0000:ffff6000       .debug$S                   0000000180000000     kernel32:KERNEL32.dll
 0000:ffff6000       .debug$S                   0000000180000000     kernel32:KERNEL32.dll
 0000:ffff6000       .debug$S                   0000000180000000     kernel32:KERNEL32.dll
 0000:ffff6000       .debug$S                   0000000180000000     kernel32:KERNEL32.dll
 0000:ffff6000       .debug$S                   0000000180000000     kernel32:KERNEL32.dll
 0000:ffff6000       .debug$S                   0000000180000000     kernel32:KERNEL32.dll
 0000:ffff6000       .debug$S                   0000000180000000     kernel32:KERNEL32.dll
 0000:ffff6000       .debug$S                   0000000180000000     kernel32:KERNEL32.dll
 0000:ffff6000       .debug$S                   0000000180000000     kernel32:KERNEL32.dll
 0000:ffff6000       .debug$S                   0000000180000000     wsock32:WSOCK32.dll
 0001:00000644       ConstructTicketRequest     0000000180001644 f   NativeCreds.obj
 0001:000015d0       $$000000                   00000001800025d0     MSVCRT:amdsecgs.obj
 0001:00001600       ?dllmain_crt_dispatch@@YAHQEAUHINSTANCE__@@KQEAX@Z 0000000180002600 f   MSVCRT:dll_dllmain.obj
 0001:00001650       ?dllmain_crt_process_attach@@YAHQEAUHINSTANCE__@@QEAX@Z 0000000180002650 f   MSVCRT:dll_dllmain.obj
 0001:00001768       ?dllmain_crt_process_detach@@YAH_N@Z 0000000180002768 f   MSVCRT:dll_dllmain.obj
 0001:000017ec       ?dllmain_dispatch@@YAHQEAUHINSTANCE__@@KQEAX@Z 00000001800027ec f   MSVCRT:dll_dllmain.obj
 0001:00001a68       capture_previous_context   0000000180002a68 f   MSVCRT:gs_report.obj
 0001:00002310       $$000000                   0000000180003310     MSVCRT:guard_dispatch.obj
 0001:00002330       $$000000                   0000000180003330     MSVCRT:guard_xfg_dispatch.obj
 0001:00002346       ?fin$0@?0??dllmain_crt_process_attach@@YAHQEAUHINSTANCE__@@QEAX@Z@4HA 0000000180003346 f   MSVCRT:dll_dllmain.obj
 0001:0000235d       ?fin$0@?0??dllmain_crt_process_detach@@YAH_N@Z@4HA 000000018000335d f   MSVCRT:dll_dllmain.obj
 0001:00002376       ?fin$1@?0??dllmain_crt_process_detach@@YAH_N@Z@4HA 0000000180003376 f   MSVCRT:dll_dllmain.obj
 0001:0000238a       ?filt$0@?0??dllmain_dispatch@@YAHQEAUHINSTANCE__@@KQEAX@Z@4HA 000000018000338a f   MSVCRT:dll_dllmain.obj
 0001:000023c0       __scrt_is_nonwritable_in_current_image$filt$0 00000001800033c0 f   MSVCRT:utility.obj
 0002:00000df0       GS_ExceptionPointers       0000000180004df0     MSVCRT:gs_report.obj
 0002:00001348       $unwind$swprintf           0000000180005348     NativeCreds.obj
 0002:00001358       $unwind$printf             0000000180005358     NativeCreds.obj
 0002:00001364       $unwind$JNI_OnLoad         0000000180005364     NativeCreds.obj
 0002:00001378       $unwind$JNI_OnUnload       0000000180005378     NativeCreds.obj
 0002:00001378       $unwind$__scrt_initialize_default_local_stdio_options 0000000180005378     MSVCRT:default_local_stdio_options.obj
 0002:00001378       $unwind$?dllmain_crt_dispatch@@YAHQEAUHINSTANCE__@@KQEAX@Z 0000000180005378     MSVCRT:dll_dllmain.obj
 0002:00001378       $unwind$DllMain            0000000180005378     MSVCRT:dll_dllmain_stub.obj
 0002:00001378       $unwind$__GSHandlerCheck   0000000180005378     MSVCRT:gshandler.obj
 0002:00001378       $unwind$__scrt_acquire_startup_lock 0000000180005378     MSVCRT:utility.obj
 0002:00001378       $unwind$__scrt_dllmain_after_initialize_c 0000000180005378     MSVCRT:utility.obj
 0002:00001378       $unwind$__scrt_dllmain_before_initialize_c 0000000180005378     MSVCRT:utility.obj
 0002:00001378       $unwind$__scrt_dllmain_crt_thread_attach 0000000180005378     MSVCRT:utility.obj
 0002:00001378       $unwind$__scrt_dllmain_crt_thread_detach 0000000180005378     MSVCRT:utility.obj
 0002:00001378       $unwind$__scrt_dllmain_uninitialize_c 0000000180005378     MSVCRT:utility.obj
 0002:00001378       $unwind$__scrt_dllmain_uninitialize_critical 0000000180005378     MSVCRT:utility.obj
 0002:00001380       $unwind$Java_sun_security_krb5_Credentials_acquireDefaultNativeCreds 0000000180005380     NativeCreds.obj
 0002:000013a4       $unwind$PackageConnectLookup 00000001800053a4     NativeCreds.obj
 0002:000013b4       $unwind$ConstructTicketRequest 00000001800053b4     NativeCreds.obj
 0002:000013d0       $unwind$ConcatenateUnicodeStrings 00000001800053d0     NativeCreds.obj
 0002:000013d0       $unwind$_DllMainCRTStartup 00000001800053d0     MSVCRT:dll_dllmain.obj
 0002:000013e0       $unwind$BuildTicket        00000001800053e0     NativeCreds.obj
 0002:000013f8       $unwind$BuildPrincipal     00000001800053f8     NativeCreds.obj
 0002:00001414       $unwind$BuildEncryptionKey 0000000180005414     NativeCreds.obj
 0002:00001428       $unwind$BuildTicketFlags   0000000180005428     NativeCreds.obj
 0002:00001438       $unwind$BuildKerberosTime  0000000180005438     NativeCreds.obj
 0002:00001458       $unwind$ThrowOOME          0000000180005458     NativeCreds.obj
 0002:00001458       $unwind$_RTC_Initialize    0000000180005458     MSVCRT:initsect.obj
 0002:00001458       $unwind$_RTC_Terminate     0000000180005458     MSVCRT:initsect.obj
 0002:00001464       $unwind$ShowLastError      0000000180005464     NativeCreds.obj
 0002:00001470       $unwind$Java_sun_security_krb5_Config_getWindowsDirectory 0000000180005470     WindowsDirectory.obj
 0002:00001484       $unwind$__GSHandlerCheckCommon 0000000180005484     MSVCRT:gshandler.obj
 0002:00001490       $xdatasym                  0000000180005490     MSVCRT:amdsecgs.obj
 0002:00001494       $unwind$?dllmain_crt_process_attach@@YAHQEAUHINSTANCE__@@QEAX@Z 0000000180005494     MSVCRT:dll_dllmain.obj
 0002:000014d0       $unwind$?fin$0@?0??dllmain_crt_process_attach@@YAHQEAUHINSTANCE__@@QEAX@Z@4HA 00000001800054d0     MSVCRT:dll_dllmain.obj
 0002:000014d0       $unwind$?fin$0@?0??dllmain_crt_process_detach@@YAH_N@Z@4HA 00000001800054d0     MSVCRT:dll_dllmain.obj
 0002:000014d0       $unwind$?fin$1@?0??dllmain_crt_process_detach@@YAH_N@Z@4HA 00000001800054d0     MSVCRT:dll_dllmain.obj
 0002:000014d8       $unwind$?dllmain_crt_process_detach@@YAH_N@Z 00000001800054d8     MSVCRT:dll_dllmain.obj
 0002:0000152c       $unwind$?dllmain_dispatch@@YAHQEAUHINSTANCE__@@KQEAX@Z 000000018000552c     MSVCRT:dll_dllmain.obj
 0002:00001554       $unwind$?filt$0@?0??dllmain_dispatch@@YAHQEAUHINSTANCE__@@KQEAX@Z@4HA 0000000180005554     MSVCRT:dll_dllmain.obj
 0002:0000155c       $unwind$__report_gsfailure 000000018000555c     MSVCRT:gs_report.obj
 0002:00001564       $unwind$capture_previous_context 0000000180005564     MSVCRT:gs_report.obj
 0002:00001570       $unwind$__raise_securityfailure 0000000180005570     MSVCRT:gs_report.obj
 0002:00001570       $unwind$__scrt_initialize_crt 0000000180005570     MSVCRT:utility.obj
 0002:00001570       $unwind$__scrt_initialize_onexit_tables 0000000180005570     MSVCRT:utility.obj
 0002:00001570       $unwind$__scrt_release_startup_lock 0000000180005570     MSVCRT:utility.obj
 0002:00001570       $unwind$__scrt_uninitialize_crt 0000000180005570     MSVCRT:utility.obj
 0002:00001578       $unwind$__security_init_cookie 0000000180005578     MSVCRT:gs_support.obj
 0002:00001584       $unwind$__scrt_is_nonwritable_in_current_image 0000000180005584     MSVCRT:utility.obj
 0002:000015a4       $unwind$__scrt_is_nonwritable_in_current_image$filt$0 00000001800055a4     MSVCRT:utility.obj
 0002:000015ac       $unwind$__scrt_dllmain_exception_filter 00000001800055ac     MSVCRT:utility.obj
 0002:000015c0       $unwind$__scrt_fastfail    00000001800055c0     MSVCRT:utility_desktop.obj
 0002:000015d0       $unwind$__isa_available_init 00000001800055d0     MSVCRT:cpu_disp.obj
 0002:000015e0       $xdatasym                  00000001800055e0     MSVCRT:guard_dispatch.obj
 0002:000015e8       $xdatasym                  00000001800055e8     MSVCRT:guard_xfg_dispatch.obj
 0002:000015f0       .edata                     00000001800055f0     w2k_lsa_auth.exp
 0002:00001618       rgpv                       0000000180005618     w2k_lsa_auth.exp
 0002:00001628       rgszName                   0000000180005628     w2k_lsa_auth.exp
 0002:00001638       rgwOrd                     0000000180005638     w2k_lsa_auth.exp
 0002:00001640       szName                     0000000180005640     w2k_lsa_auth.exp
 0002:00001651       $N00001                    0000000180005651     w2k_lsa_auth.exp
 0002:0000165c       $N00002                    000000018000565c     w2k_lsa_auth.exp
 0002:00001669       $N00003                    0000000180005669     w2k_lsa_auth.exp
 0002:0000169b       $N00004                    000000018000569b     w2k_lsa_auth.exp
 0002:00001960       .idata$6                   0000000180005960     advapi32:ADVAPI32.dll
 0002:000019dc       .idata$6                   00000001800059dc     Secur32:Secur32.dll
 0002:00001a9e       .idata$6                   0000000180005a9e     kernel32:KERNEL32.dll
 0002:00001aac       .idata$6                   0000000180005aac     wsock32:WSOCK32.dll
 0002:00001b04       .idata$6                   0000000180005b04     vcruntime:VCRUNTIME140.dll
 0002:00001c22       .idata$6                   0000000180005c22     ucrt:api-ms-win-crt-string-l1-1-0.dll
 0002:00001c44       .idata$6                   0000000180005c44     ucrt:api-ms-win-crt-stdio-l1-1-0.dll
 0002:00001c64       .idata$6                   0000000180005c64     ucrt:api-ms-win-crt-runtime-l1-1-0.dll
 0003:000000c0       ?szMsgBuf@?1??ShowLastError@@9@9 00000001800060c0     NativeCreds.obj
 0003:000002c0       ?__proc_attached@@3HA      00000001800062c0     MSVCRT:dll_dllmain.obj
 0003:000002d0       GS_ExceptionRecord         00000001800062d0     MSVCRT:gs_report.obj
 0003:00000370       GS_ContextRecord           0000000180006370     MSVCRT:gs_report.obj
 0003:00000868       ?is_initialized_as_dll@@3_NA 0000000180006868     MSVCRT:utility.obj
 0003:00000869       ?module_local_atexit_table_initialized@@3_NA 0000000180006869     MSVCRT:utility.obj
 0003:00000870       ?module_local_atexit_table@@3U_onexit_table_t@@A 0000000180006870     MSVCRT:utility.obj
 0003:00000888       ?module_local_at_quick_exit_table@@3U_onexit_table_t@@A 0000000180006888     MSVCRT:utility.obj
 0005:00000060       $R000000                   0000000180008060     w2k_lsa_auth.dll.res
